:1000000008308A00FC2B0000FF00030E8301A100D2
:100010007F08A0000A08A8008A01A00E0408A20018
:100020007708A3007808A4007908A5007A08A6003C
:100030007B08A700831383128B1E20280B193328FB
:10004000220884002308F7002408F8002508F90096
:100050002608FA002708FB0028088A00210E8300E2
:10006000FF0E7F0E09008A11E9290A108A100A1171
:100070008207733431346A3429343F343E343C349B
:100080003834303420342134233427342F340134AD
:100090002A340134313468344C3456340634113443
:1000A00015340934023414340B34103404341E343F
:1000B0000D341234073405340F3416341B340A342B
:1000C000083403340C3418340E3419341D3413340A
:1000D0000A108A100A1182072034743469346D348E
:1000E00065342034283425346C34753429343A345A
:1000F000203400340A108A100A1182072034743424
:100100006F346E3465342034283425346C347534BF
:1001100029343A34203400340A108A100A11820734
:1001200020344D3473346734203428342534533428
:1001300029343A34203400340A108A100A11820714
:100140000D340A344134753474346F3420344334FC
:10015000573420344934443420342834253443344B
:1001600029343A34203400340A108A100A118207E4
:100170000D340A34433457342034533470346534E6
:1001800065346434203428342534553429343A34E1
:10019000203400340A108A100A1182070D340A3400
:1001A00049344434203461347534643469346F34F0
:1001B00000340A108A100A1182070D340A345234AE
:1001C0006534703465346134743465347234203489
:1001D0006D346F346434653420342834253443342A
:1001E00029343A34203400340A108A100A11FB3EB4
:1001F00003188A0A82000D340A3443346F3475348C
:100200007234743465347334793420346234653430
:100210006534703400340A148A100A1182070D34D0
:100220000A3443346F34753472347434653473343F
:100230007934203462346534653470342034643465
:1002400065346C346134793400340A148A100A112C
:1002500082070D340A3443346F3475347234743485
:1002600065347334793420346234653465347034E1
:1002700020346D3475346C3474342034283425348F
:10028000753429343A34203400340A148A100A119F
:1002900082070D340A3442346534613463346F3478
:1002A0006E3400340A148A100A1182070D340A349D
:1002B0005034543454342034683461346E346734E8
:1002C00000340A148A100A1182070D340A3450349B
:1002D0005434543420346D346134783400340A1486
:1002E0008A100A1182070D340A3449344434003428
:1002F0000A148A100A1182070D340A3459346534FD
:100300006C346C346F34773400340A148A100A1158
:1003100082070D340A3442346C3469346E346B34E1
:1003200000340A148A100A1182070D340A34533437
:1003300050344134433445342034773469346C3498
:100340006C342034643465346C346534743465340E
:10035000203449344434203473347434723469346E
:100360006E3467342E340D340A3449344434003446
:100370000A148A100A1182070D340A3441346C348D
:100380007434653472346E346134743465340034DA
:100390000A148A100A1182070A340D340A344E34C2
:1003A00030345834413453342034493444342D34B7
:1003B0004F342D344D346134743469346334203413
:1003C0005634253475342E34253475340A340D34BE
:1003D000003410300317A707003003180130A807B6
:1003E000003003180130A907A908031D092A2808AD
:1003F0000E3C0318A82AFF3A031D092A2708413C8E
:100400000318A82AFF3A031D092A2608403C0318AE
:10041000A82A4030A6024230031C4330A7020F3006
:10042000031C1030A8020030031C0130A902031382
:100430006F08593C031D202A0317AA1F302A0313F3
:10044000F508031D262AF60803192E2A0317AB10F8
:1004500075080319F603F503302A03130317AB14C9
:1004600083160313670F372A680F372A3A2AE70AD9
:100470000319E80AF10803193E2AF103831203174E
:10048000A408031D462AA50803194F2A24080319A6
:10049000A503A40324082504031D4F2A2A17831645
:1004A0000313610862040319662A76086202031CBA
:1004B000662A031D5F2A610875020318662A8312E3
:1004C00003172A14AA14AA118316031363086404D9
:1004D00003197B2A76086402031C7B2A031D742AF5
:1004E0006308750203187B2A831203172A14AA14BF
:1004F000AA158316031306128312061203172A1C69
:10050000872A83160313061283120616031783160F
:1005100003138612831286120317AA1C952A8316C8
:1005200003138612831286160317AA1DA82A2A1DF2
:10053000A12A8316031386128312861603172A1123
:10054000A82A8316031386128312861203172A150C
:1005500003130B118A112028031740088316031375
:100560009B009C131C141A08F80083120034031714
:100570003908C0000313AC220317BB017808BA0086
:1005800001303907BC00C0000313AC220030031750
:10059000BA070318BB0A7808BB073A08F8003B08FB
:1005A000F9000313003403174508F8014402031847
:1005B000DC2A4408F700E82AF7010830C600C40D19
:1005C000F70D450877020318F700F80DC60BDF2A70
:1005D00003130034780803174208C4006430C500D0
:1005E0000313D32277080317C20078083030031DA5
:1005F000002B43180B2BC3190B2B431A2030022B53
:10060000C3114312F807780803130C1A092B0317B8
:10061000042B990003174208C4000A30C5000313D5
:10062000D32277080317C20078083030031D1C2B33
:10063000C319252B431A2030F807780803130C1A26
:10064000232B03171E2B990003173030C2074208D3
:1006500003130C1A2D2B0317282B99000034453057
:100660008400831700080319442B0130F800F701B8
:10067000F70B382BF80B372B4A30F700F70B3E2BD4
:1006800000000000800B352B00340317BE013E082C
:10069000043C031C562B83160313650883120317AF
:1006A000C50003132F230317BE0A472B031300347F
:1006B000F801F901F701FA0103174B08031D632B39
:1006C0004A0803197D2B1030CC000310C80DC90D4A
:1006D000F70DFA0D4B087A02031D702B4A087702BA
:1006E000031C792B4A08F702031CFA034B08FA0291
:1006F0000314F80DF90DCC0B652B00000313003427
:100700000317C0080319E12B0430C900B030C8003A
:10071000CB0103136E080317CA000313582379088B
:100720008316E6007808E5000030F80006388312EA
:1007300092000317200883160313920083120317F5
:10074000210CC600200CC500C60CC50C3F30C605E8
:10075000C60CC50CC60CC50CC60C45080313950089
:100760000317C60C460C3039F70003131708CF39AE
:1007700077049700831686118312861583168510D9
:10078000831285140317C101400841020318D32BBB
:1007900083160313650883120317C50003132F2361
:1007A0000317C10AC42B8316031385108312851007
:1007B00083168615650883120317C50003132F23BC
:1007C00003170313003403173E0BE72BF32BBF0172
:1007D0000310BE0CBF0D0314BF0D3F08C000031370
:1007E0008023E32B0317BF013F08013C031C032CAC
:1007F00083160313650883120317C50003132F2301
:100800000317BF0AF42B03138A11242C03173C0887
:10081000203C031D0F2C03134523242C0317013008
:10082000BD003C082B3C0318202C3C085A3C031C00
:10083000202C2C303C0203133520F8000317BD0098
:100840003D08BE000313E32B003478080317390872
:10085000C4006430C5000313D32277080317B9001E
:1008600078083030031D3B2C3A18432CBA19432C1E
:100870003A1A20303D2CBA113A12F8077808BC0019
:100880000313062403173908C4000A30C5000313F4
:10089000D32277080317B90078083030031D542C91
:1008A000BA195A2C3A1A2030F8077808BC000313FA
:1008B000062403173030B9073908BC000313062497
:1008C000003483160510831205140317AA1A6D2C21
:1008D000AA162308A5002208A40003130034F70178
:1008E000F80103173F0803104018F707F70CF80C3E
:1008F000C018F707F70CF80C4019F707F70CF80CBD
:10090000C019F707F70CF80C401AF707F70CF80CAA
:10091000C01AF707F70CF80C401BF707F70CF80C98
:10092000C01BF707F70CF80C03138A11242D83164C
:100930000510831205100317AA12A501A4010313C1
:1009400000340317B9080319A82C3908BA00E22C9F
:10095000AB1CC12C83160313061483120618BD2C7E
:1009600094300317C0000313AC22F8080319BD2C00
:1009700094300317BA00C02C031314300317BA00C5
:10098000E22C5430C0000313AC22F8080319CD2C1C
:1009900054300317BA00E22C031383160614831293
:1009A0000618DF2C94300317C0000313AC22F8089C
:1009B0000319DF2C94300317BA00E22C0313143010
:1009C0000317BA002A14AA11AA10831603130617D4
:1009D0008312061BED2C0317E52C61240830031746
:1009E000BC00FA30C50003132F230317BC0BF12CF6
:1009F0003A08BA0ABC00C0000313AC2278080317F7
:100A0000BB00BB0803198B2D3B083A3C03190E2D84
:100A10003B08BC0003130624892D03173A08BC00C9
:100A2000BD013C08BC0ABF00C0000313AC2278081B
:100A30000317BE003E083A3C03192A2D3D08BF00AB
:100A40000A30C00003136F2C78080317BD00303044
:100A50003E02BD073E083A3C031D112D3D08F8003B
:100A60007808BB000030F800063803139200031723
:100A7000200883160313920083120317210CBD0074
:100A8000200CBC00BD0CBC0C3F30BD05BD0CBC0C2B
:100A9000BD0CBC0CBD0C3C08031395000317BD0C2A
:100AA0003D0C3039F70003131708CF39770497004E
:100AB000831686118312861583168510831285147A
:100AC00004300317BC00FA30C50003132F230317AB
:100AD000BC0B632DBB0303196F2D0313602D83160D
:100AE000031385108312851083168615831203174E
:100AF0003A08BA0ABC00C0000313AC2278080317F6
:100B0000BB003B083A3C0319882D83160313762D4E
:100B100003130317F82C6430C50003132F23831627
:100B200086178312861F952D972403172A10AA145F
:100B3000AA11AA1383160313E801E7017D08F60042
:100B40007C08F50083120317AB10031300348C1ECE
:100B5000A72D1808A9001A08F800A91CB12D181211
:100B60001816000000340317D2010408D1005210F7
:100B7000831B52144B0EF038CD00CD07E23ECE0061
:100B8000323ED0004B080F39CE07CE07D007E93EE2
:100B9000CF00CF07CF074A0E0F39CF07D007CF0DB1
:100BA000D00DD009D00D4A080F39D007CD0D073030
:100BB000CC000A30D007CF03031CDA2DCF07CE03B9
:100BC000031CDE2DCE07CD03031CE22DCD07CC0385
:100BD000031CE62D4C308400831707305105840731
:100BE0005030040203190C2E0008F700031DFE2DDF
:100BF000511A0A2ED119002E2030012E0830D100B2
:100C00003030F707770803130C1A082E0317032E4A
:100C100099000317840AF02D0008F7003030F70719
:100C2000770803130C1A162E0317112E990000349F
:100C30000317C803C9010313A72578080317CB00BE
:100C4000603C03182A2E4B087A3C031C2A2E4B08C2
:100C5000DF392B2E4B08CA004A08083C031D492ED9
:100C6000C9080319482EC9034A0803130C1A3A2E5F
:100C70000317352E990020300C1E3C2E99000317C7
:100C80004A0803130C1A462E0317412E9900031726
:100C9000662E4A081F3C0318662E4A087E3C031C39
:100CA000662E480849020318662E4908C90A4607F5
:100CB00084008313471883174A0880004A080313E7
:100CC0000C1A642E03175F2E990003174A080D3C77
:100CD000031D1B2E490846078400831347188317FA
:100CE0008001031300348C1E732E0317C701A0303C
:100CF000C6000630C8000313182600341030F70071
:100D0000FA010317D301D00CCF0C031C8D2E510810
:100D1000FA070318D30A5208D307D30CFA0CF90CBC
:100D2000F80CF70B832E03138A11BB2E0317C9018E
:100D3000CA01CC01CE01A030CD004D084E040319EC
:100D4000AA2E4C08CC0A4D07840083134E18831733
:100D50000008CB004B082F3C0318D22E4B08393C1F
:100D6000031CD22ED0010A30CF004A08D200490815
:100D7000D10003137E2E79080317D0007808CF0026
:100D800030304B024F07C9005008CA000318CA0A86
:100D90004C08CC0A4D07840083134E1883170008B3
:100DA000CB00AA2E4908F8004A08F90003130034C2
:100DB00003174B08831603139B00831203174C0879
:100DC000831603139A001C1583120B08F7008B136C
:100DD000831655309D00AA309D009C149C18EE2E61
:100DE0001C11770883128B0400340130FA0047305D
:100DF000840083137A18831700080317C900460874
:100E0000CB004908CC000313D8260130031746074E
:100E1000C9000130FA004830840083137A18831720
:100E20000008CA004908CB004A08CC000313D826A2
:100E300000340317C5014508031368200317C50ACA
:100E4000F70003130C1A262F0317212F99000730E0
:100E500003174502031D1B2F103084004308CB00ED
:100E60004208CA000313B32529300C1E352F990000
:100E70003A300C1E392F990020300C1E3D2F99005E
:100E8000732601300317C6004230C50083160313D2
:100E9000A00803195F2F8312962679080317C8004C
:100EA0007808C70045088400831346188317840A0E
:100EB00048088000840347088000831603138312C8
:100EC0000317C40803196E2F4108C6004308C80061
:100ED0004208C7000313F526742F03174108CB00FF
:100EE0004208CC000313D82600340317BC013C0889
:100EF00003139C200317BC0AF70003130C1A822F5C
:100F000003177D2F99000E3003173C02031D772F26
:100F100003136D080C1E8A2F990029300C1E8E2F8A
:100F200099003A300C1E922F990020300C1E962FFB
:100F3000990073268316A0080319AD2F2008593C89
:100F4000031DA72F59308312ED00AE2F83164E30AC
:100F50008312ED008316EA01E90183120E300317B4
:100F6000CB0003136D080317CC000313D8268A1592
:100F7000F52B03172A1FDA2F5430BC000313062465
:100F80004F300317BC000313062454300317BC0072
:100F9000031306244523F601F5010317AB14B90129
:100FA0000313A1249724831686178312861FD32F39
:080FB00003172A130313003498
:101000000317BD013D083F3C031C18282C303D0749
:10101000840083133D083C07C000831603139B0024
:101020009C131C141A08800083120317BD0A02289F
:10103000BE013E088A1103138C208A150317BE0ACD
:10104000F70003130C1A26280317212899000630ED
:1010500003173E02031D19282C308400831300302F
:10106000000403193D2803130C1A382803173328EA
:1010700000089900840A03172F28293003130C1A3B
:10108000432803173E2899003A300C1E4528990042
:1010900020300C1E492899008C1E4C280317C701CC
:1010A000A030C6004030C8008A11031318268A15E4
:1010B0008316A008031993282008203C031D6328E9
:1010C000A001EA01E90183120317BD013D083F3C7D
:1010D000031C91283D083C07BE00A0303D0784005A
:1010E00083130008BF003E08CB003F08CC008A11E4
:1010F0000313D8268A152C3003173D07BE00BF0105
:101100000318BF0AA0303D07840083130008C00005
:101110003E08840083133F18831740088000BD0AEF
:101120006628831603138312003401300317420725
:10113000C6004308C7000318C70AF430C9002430AA
:10114000C8004708CB004608CA008A110313582379
:101150008A1579080317C8007808C700C90149082B
:101160008A1103137A208A150317C90AF70003139B
:101170000C1ABC280317B728990007300317490237
:10118000031DAF28103084004808CB004708CA0070
:101190008A110313B3258A1529300C1ECD28990016
:1011A0003A300C1ED128990020300C1ED528990009
:1011B0008A1173268A158316A008031932298A1109
:1011C000831296268A1579080317C5007808C4008B
:1011D0004508C7004408C60047080C3C0318FB2814
:1011E000FF3A031DF7284608AC3C0318FB280D30D6
:1011F000C700AC30C600C708031D05294608F93CE6
:10120000031C0529C701FA30C6004608F800470844
:10121000F9007908C5007808C400F430C90024300A
:10122000C8004508CB004408CA008A11031358239C
:101230008A1579080317C7007808C60001304602EE
:10124000C2004708C3000030031C0130C30241083C
:10125000C6004308C8004208C7008A110313F526D8
:101260008A158316831200340317BC01BD01BE0129
:101270003E088A110313B4208A150317BE0AF7002B
:1012800003130C1A45290317402999000C30031742
:101290003E02031D382903136E080317C2001830DD
:1012A000C3008A110313EA228A1529300C1E56291D
:1012B00099003A300C1E5A29990020300C1E5E29E4
:1012C00099008A1173268A158A1196268A1579083B
:1012D0000317BD007808BC003C083D0403197F29B2
:1012E0003C080313EE000F300317CB0003136E0806
:1012F0000317CC008A110313D8268A150317BE01E1
:101300003E088A110313CA208A150317BE0AF70084
:1013100003130C1A8D290317882999000A30031723
:101320003E02031D80290830C100831603136E0896
:1013300083120317C300831603136D088312031768
:10134000C200031395208A15F72B0317BC01BD01BA
:10135000BE01BF01C10141088A110313D9208A15BA
:101360000317C10AF70003130C1AB8290317B3298E
:101370009900113003174102031DAB2903136F08B5
:101380000C1EC029990029300C1EC42999003A303E
:101390000C1EC829990020300C1ECC2999008A11F6
:1013A00073268A158316A0080319052A2008593CBC
:1013B000031DDF2959308312EF00F92983164E30BF
:1013C0008312EF008316EA01E9010230831203174A
:1013D000C600831603136A0883120317C800831616
:1013E0000313690883120317C7008A110313F52634
:1013F0008A1510300317CB0003136F080317CC00B6
:101400008A110313D8268A15831683126F08593C54
:10141000031D292B83166B086C0403192F2A013036
:101420006B07F8006C08FA000318FA0A78088312B0
:101430000317C1007A08C200F430C9002430C80084
:101440004208CB004108CA008A11031358238A15A9
:1014500079080317BF007808BE00831603138312B0
:101460000317C10141088A110313F4208A150317D9
:10147000C10AF70003130C1A3F2A03173A2A9900EE
:101480000F3003174102031D322A0A30C1008316B0
:1014900003136C0883120317C300831603136B082E
:1014A00083120317C200031395200317C1014108DB
:1014B0008A1103130B218A150317C10AF7000313BE
:1014C0000C1A642A03175F2A99001530031741028A
:1014D000031D572A1330C100C3017408C200C401A0
:1014E0008A11031319278A150317C10141088A11AC
:1014F000031325218A150317C10AF70003130C1AD9
:10150000832A03177E2A9900163003174102031D10
:10151000762A7308C2001830C3008A110313EA2226
:101520008A1529300C1E922A99003A300C1E962AF0
:10153000990020300C1E9A2A99008A1173268A1568
:101540008316A0080319BF2A8A11831296268A15CA
:1015500079080317BD007808BC00BD08031DB62A32
:101560003C08633C031CB62A3C08F3001230CB0055
:101570007308CC008A110313D8268A1583168312A8
:101580000317C10141088A11031345218A15031766
:10159000C10AF70003130C1ACF2A0317CA2A9900AD
:1015A000083003174102031DC22A0230C10083160E
:1015B00003136A0883120317C30083160313690811
:1015C00083120317C2000130C4008A1103131927C4
:1015D0008A150317C10141088A11031352218A1584
:1015E0000317C10AF70003130C1AF82A0317F32A8A
:1015F00099000A3003174102031DEB2A1130C10084
:10160000C3017208C200C4018A11031319278A1585
:101610000317C10141088A11031361218A150317B9
:10162000C10AF70003130C1A172B0317122B99008A
:10163000093003174102031D0A2B0C30C100230897
:10164000C3002208C2000130C4008A110313192705
:101650008A158A15F82B0317B9018316031386120E
:101660008312861283160612831206160317BC0114
:101670003C088A1103136F218A150317BC0AF7006F
:1016800003130C1A452B0317402B99000430031742
:101690003C02031D382BC1017D08C3007C08C20039
:1016A0000130C4008A11031319278A150317BC01DE
:1016B0003C088A11031378218A150317BC0AF70026
:1016C00003130C1A652B0317602B990008300317BE
:1016D0003C02031D582B0430C1008316031362081B
:1016E00083120317C30083160313610883120317C1
:1016F000C2000130C4008A11031319278A15031789
:10170000BC013C088A11031385218A150317BC0A02
:10171000F70003130C1A8E2B0317892B990007303F
:1017200003173C02031D812B0630C10083160313EF
:10173000640883120317C30083160313630883121C
:101740000317C2000130C4008A11031319278A1538
:101750000317BC013C088A11031391218A15031752
:10176000BC0AF70003130C1AB72B0317B22B99000E
:10177000223003173C02031DAA2B1430BC000313B4
:1017800000200317BC013C088A11031345218A1568
:101790000317BC0AF70003130C1AD02B0317CB2B2B
:1017A0009900083003173C02031DC32B5430BC00C2
:1017B000031300200317BC013C088A110313B8214E
:1017C0008A150317BC0AF70003130C1AE92B031739
:1017D000E42B99000B3003173C02031DDC2B9430E3
:1017E000BC00031300208A11752F8A153429A529FE
:1017F0008A0100288A15FC2D840183131F3083057C
:1018000007309F00193083169900263098009030D9
:1018100083129800A901AA01AB0107309F0083162B
:1018200005080330F700F70B132C83121F080C1365
:1018300083168113061283120612831686128312F0
:1018400086128316051083120510831685108312E5
:10185000851083160108C03903388100B530831222
:10186000900007309F00831605080330F700F70B40
:10187000372C83121F080C1383169F018312031742
:10188000AB01AA0103138B160317B9018A110313C5
:10189000B7228A157908FD007808FC000430031788
:1018A000B9008A110313B7228A1579088316E2005A
:1018B0007808E100063083120317B9008A11031378
:1018C000B7228A1579088316E4007808E30002300D
:1018D00083120317B9008A110313B7228A157908F6
:1018E0008316EA007808E9000C3083120317B90068
:1018F0008A110313B7228A1579080317A300780801
:10190000A2000A30B9008A110313B7228A15790898
:101910008316EC007808EB00083083120317B90037
:101920008A110313B7228A1579088316EE00780806
:10193000ED000E3083120317C0008A110313AC228E
:101940008A157808ED000F300317C0008A110313C1
:10195000AC228A157808EE0010300317C0008A11F7
:101960000313AC228A157808EF0011300317C0006A
:101970008A110313AC228A157808F200123003177B
:10198000C0008A110313AC228A157808F3001330C3
:101990000317C0008A110313AC228A157808F400DB
:1019A00083168611831286110C30970083168615D4
:1019B0006E0883120317A100831603136D088312A8
:1019C0000317A0000030F800063803139200031735
:1019D00020088316031392007D08F6007C08F500AA
:1019E00083120317A901A801A701A601AB01AA014F
:1019F000F0017D0883160313E8007C08E70000303F
:101A00008500831285016500C0308B040317B9017E
:101A100039088A110313C8218A150317B90AF70078
:101A200003130C1A152D0317102D990015300317E9
:101A30003902031D082D0230C2001830C3008A117C
:101A40000313EA228A152E300C1E242D99000A3029
:101A50000317C2001830C3008A110313EA228A1543
:101A60000A300C1E312D99000D300C1E352D9900B9
:101A70000317AA1483160313061483120618CC2D19
:101A800056300317BC008A11031306248A1502304E
:101A90000317B9001830BA008A11031325248A15D8
:101AA0002E300317BC008A11031306248A150A304E
:101AB0000317B9001830BA008A11031325248A15B8
:101AC00020300317BC008A11031306248A152F3017
:101AD0000317BC008A11031306248A158A114523B3
:101AE0008A1514300317C0008A110313AC228A151B
:101AF000F808031D8F2D54300317C0008A110313FB
:101B0000AC228A15F808031D8F2D94300317C000EE
:101B10008A110313AC228A15F8080319CC2D14304E
:101B20000317B9008A110313A1248A15543003172F
:101B3000C0008A110313AC228A15F8080319B12DCD
:101B40008A1145238A152F300317BC008A1103130D
:101B500006248A1554300317B9008A110313A124EF
:101B60008A1594300317C0008A110313AC228A151A
:101B7000F8080319CC2D8A1145238A152F30031735
:101B8000BC008A11031306248A1594300317B90088
:101B90008A110313A1248A158C1EFF2D0317AC0193
:101BA0008A110313A7258A1578080317AD002D089D
:101BB0000D3C0319DF2D2D080A3C031DFE2D2C08BA
:101BC000AC0A133C031CFE2DFA30C5008A11031326
:101BD0002F238A158C1EFC2D8A11A7258A157808BB
:101BE0000317AD002D080D3C0319FA2D2D080A3CF2
:101BF000031DFD2D03132B2B0317DF2D03136F087C
:101C0000593C031D8A2E831686178312861B2D2EA0
:101C10008A1161248A150317AA15AA172B107D08AB
:101C2000831603136802031C202E031D1B2E670856
:101C30007C020318202EF6010A30F500E801E701C6
:101C400083120B138B138B1B222E7208F100C030F2
:101C50008B048A11B9278A158A2E0317AA1E802E93
:101C6000F3080319802E2B18802EAD0174082D0265
:101C700003184F2E6430C5008A1103132F238A15D1
:101C8000831686178312861B4B2E01300317B00074
:101C90004F2E4D2E03130317B001AD0A362EB00898
:101CA000031D802E831603136C0883120317A100F3
:101CB000831603136B0883120317A0007308C00078
:101CC0008A11031380238A1583166E088312031763
:101CD000A100831603136D0883120317A0000313DA
:101CE0000B138B138B1B712E03172308A5002208DF
:101CF000A4007208F100C03003138B0403172B14E7
:101D0000F108031D892E8A11031397248A150317DE
:101D10002B1003136D084E3C031DBB2E0317AB1C89
:101D2000B92E8316031386128312861283160612A7
:101D3000831206160317AE012E08093C031CB12EB0
:101D40008316031305108312051403106E0C03177A
:101D5000B900C0008A11031380238A150317AE0A45
:101D60009C2E831603130510831205108A01002888
:101D70000317152F03130317AB18D52E8316031360
:101D8000E908031DC62EEA080319172F6A0868021E
:101D9000031C172F0319CF2E83120317D52E6908A2
:101DA0006702031C172F83120317AA11831603134C
:101DB0008612831286128316061283120616831663
:101DC00086178312861BF82E831668087D02031877
:101DD000EB2E8312F82E031DF32E7C086702031CE2
:101DE000F32E8312F82E8A118312B9278A15DF2E5B
:101DF0000317B9018A110313A1248A1508300317A8
:101E0000B900FA30C5008A1103132F238A1503176E
:101E1000B90B012F831603130612831206128316C1
:101E20008612831286160317AA13831603138312CE
:041E3000CC2D630052
:1042000058000200000000003C0000001E000000FA
:104210005200000052000000000000004E000F009D
:0A4220004E00000001000500000040
:0242A800000014
:02432800000093
:02400E00223F4F
:00000001FF
